:1000000028200020510100004D0100004D0100009A
:1000100000000000000000000000000000000000E0
:100020000000000000000000000000004D01000082
:1000300000000000000000004D0100004D01000024
:100040004D0100004D0100004D0100004D01000078
:100050004D0100004D0100004D0100004D01000068
:100060004D0100004D0100004D0100004D01000058
:100070004D0100004D0100004D0100004D01000048
:100080004D0100004D0100004D0100004D01000038
:100090004D0100004D0100004D0100004D01000028
:1000A0004D0100004D0100004D0100004D01000018
:1000B000000000000448054B10B5834203D0044BF8
:1000C000002B00D0984710BD9C0600009C06000045
:1000D0000000000006480749091A8B10C90FC9180B
:1000E00010B5491003D0044B002B00D0984710BD29
:1000F0009C0600009C0600000000000010B5074CA4
:100100002378002B09D1FFF7D5FF054B002B02D038
:10011000044800E000BF0123237010BD0000002050
:10012000000000009C060000054B10B5002B03D01A
:100130000449054800E000BFFFF7CCFF10BDC046F2
:1001400000000000040000209C060000FEE7000004
:100150002449254870B581420AD0244BC41E002290
:10016000A34203D303331A1A92089200204B9847F4
:100170002048214BC11E0022994203D803331A1A8A
:100180009208920000211D4B9847FF221C4B03212F
:1001900093431C4A0C259360022208241A4B1B48E7
:1001A0005A62C3788B431343C370C378AB43234372
:1001B000C3703020164B9E7B8643103830439873B3
:1001C000987BA84304439C73987B884302439A73AB
:1001D0008023104A51680B4353600F4B98470F4BD5
:1001E0009847FEE79C060000000000200000002069
:1001F0002106000000000020280000203306000037
:100200000000000000ED00E0FC70004100500041E3
:100210000048004100400041D905000005040000ED
:10022000064B1A7AD2B21A725A7AD2B25A729A7AA1
:10023000D2B29A72DA7AD2B2DA727047000400400F
:10024000064B10B55A685A60054B9847054B9847BE
:10025000054B9847FF20054B984710BD00400041D3
:100260002102000079020000C1020000E503000045
:10027000002800D100BE70470E4B0F48196A1A6A59
:100280000140920F92070A430C490A431A62022264
:1002900099690A431F219A611A7F0A401A771E3909
:1002A000DA68D2080A42FBD08022196A0A431A622D
:1002B0007047C046000800400000FF0F0203000026
:1002C0000221024A93698B43936170470008004002
:1002D000F7B506000D001400002804D0081E02D057
:1002E0001000431E9841F1221149124B98473700E4
:1002F000114B08373800019398470028F7D00026A3
:100300003800A95D0D4B98473800019B984700289D
:10031000FAD00136B442F3D80125002C00D02500D4
:100320003800074B98470028FAD02800FEBDC04689
:100330004206000071020000AF050000A1050000A8
:10034000B9050000F7B5050014000191002804D09C
:10035000081E02D01000431E984186220C490D4B06
:100360005200984700262F00083738000A4B98475C
:100370000028F8D0094B38009847019B9855013662
:10038000B442F0D80120002C00D02000FEBDC046B1
:100390004206000071020000C3050000A70500002E
:1003A00070B504000D00002802D00800431E9841DB
:1003B0000749084B3422984720002900064B083093
:1003C0009847002803D1054B6360054B236070BD3F
:1003D000420600007102000079050000450300009C
:1003E000D1020000C00709D58023054A5B00936055
:1003F00083235B0253605378DB09FCD17047C0460E
:10040000000C004010B5014B9847FEE7CD050000F9
:100410000D4B0122180030B5443001780F24914370
:10042000114301701900032032310D784533A54383
:10043000284308701878904302431A7030230A78D2
:10044000224013430B7030BD004400410423044A92
:10045000116A0B431362034B034A5A807047C0462C
:1004600000040040000C00401440000010B5054B93
:10047000984700220449054B05489847054B984783
:1004800010BDC0464D04000000080042A10300005A
:100490001C0000201104000010B5024B9847024BCD
:1004A000984710BD410200006D040000C369194265
:1004B000FCD17047022210B5036803219343036007
:1004C000014B984710BDC046AD04000010B5016057
:1004D000014B0321984710BDAD040000F8B51B4B3C
:1004E0000400C3189B0ADBB2002B04D0002018497B
:1004F000184A194B9847E369184E194DDB0710D479
:100500000227184B03212000984723683B4205D05F
:100510002000154B984739002000B04705212000E6
:10052000A84720000121B04720001049A847C02358
:100530009B022000636007210D4B984700200D4B64
:10054000A381A07330342070F8BDC04600F8FFBD11
:100550005E0600003A02000071020000AD040000D7
:10056000CD040000AD040000B504000004001040FC
:10057000AD040000ADD8FFFF70B505000C00B4223B
:1005800004490120044B98472C602000034B9847F6
:1005900070BDC0465E06000071020000DD04000070
:1005A0000368198570470368188DC0B270470368E7
:1005B000187E0123184070470368187E8007C00F1B
:1005C00070470368187E4007C00F704710B5014B95
:1005D000984710BD9904000070B500260C4C0D4DD5
:1005E000641BA410A64209D1002600F047F80A4C6B
:1005F0000A4D641BA410A64205D170BDB300EB5890
:1006000098470136EEE7B300EB5898470136F2E71A
:1006100088060000880600008C060000880600009E
:10062000002310B59A4200D110BDCC5CC4540133F4
:10063000F8E703008218934200D170471970013324
:10064000F9E72E2E2F68616C2F7372632F68616C2F
:100650005F75736172745F73796E632E63002E2E03
:100660002F68706C2F736572636F6D2F68706C5F8D
:10067000736572636F6D2E6300000000F8B5C046AD
:10068000F8BC08BC9E46704729010000F8B5C0467A
:0C069000F8BC08BC9E467047FD0000004E
:00000001FF
